:020000020000FC
:1000000002C043C043C04FED4DBF47E147BBC29A5A
:10001000C19AC09A41E043BF42E049BF10E021E2EB
:1000200032E47894C49A0000C4980000133619F49E
:10003000E89450F904C0112311F4689450F950FB6E
:1000400016F4139501C01A95233619F4E89451F962
:1000500004C0222311F4689451F951FB16F423953E
:1000600001C02A95333619F4E89452F904C03323B9
:1000700011F4689452F952FB16F4339501C03A9585
:100080008A94F1F79A94E1F7CDCF18954CE942BFE5
:10009000043621F40027C298C198C098011708F0CF
:1000A000C29A021708F0C19A031708F0C09A039584
:0200B0001895A1
:00000001FF
